:020000040000FA
:1000000081EF07F01200FFFF04EF10F01200FFFF76
:10001000FFFFFFFFFFFFFFFF0CEF10F01200FFFFDD
:10002000FFFFFFFFFFFFFFFFFFFF01002E0F00009C
:10003000C000000002000000550EA76EAA0EA76EB9
:10004000A68212000001420E6A6F020E6B6F010E53
:100050006C6F12000001606B6651605D1EE260C053
:1000600000F0016A026A67510024F36E68510120B2
:10007000F46E69510220F86EF4CFF7FFF3CFF6FF6C
:100080000800F5CF61F06051EA6A6A0FE96E000E70
:10009000EA2261C0EFFF602BDFD7F86A1200840EFE
:1000A000A66E0001606B6651605D27E26051EA6AEE
:1000B0006A0FE96E000EEA22EFCF03F060C000F095
:1000C000016A026A67510024F36E68510120F46EE0
:1000D00069510220F86EF4CFF7FFF3CFF6FF03C0AB
:1000E000F5FF0C001F0E60151F0803E06605605D3C
:1000F00001E1A2DF0001602BD6D712000001606B86
:100100006651605D20E2940EA66E6051006E016A39
:10011000060ED89000360136E804FBE1026A01BE03
:100120000268000167510024F36E68510120F46EEB
:1001300069510220F86EF4CFF7FFF3CFF6FF7CDFB2
:100140000001602BDDD7F86A1200A66A0001606B1F
:100150006651605D0EE267516025A96EA680605110
:10016000EA6A6A0FE96E000EEA22A8CFEFFF602B61
:10017000EFD712000001606B6651605D13E26751BA
:100180006025A96E6051EA6A6A0FE96E000EEA22E4
:10019000EF50A86E040EA66E4FDFA6B2FED7000188
:1001A000602BEAD71200C40EA66E0001606B665188
:1001B000605D20E26051EA6A6A0FE96E000EEA2291
:1001C000EFCF03F060C000F0016A026A67510024BB
:1001D000F36E68510120F46E69510220F86EF4CF7D
:1001E000F7FFF3CFF6FF03C0F5FF0C0025DF00019A
:1001F000602BDDD7F86A12008150200B01E0010E60
:1002000000016A6F12000001C051C11104E1200E0B
:10021000C06F4E0EC16FC007000EC15B6DA20BD048
:10022000C051C11107E18C708C50010B02E08C822F
:1002300001D08C922FD00001B75103E18C908C92A9
:1002400029D0B70503E18C808C8224D0020EB75DE3
:1002500003E18C808C921ED0030EB75D03E18C907D
:100260008C8218D0050EB75D07E10001C051C111A5
:1002700002E18C708C920ED0060EB75D0BE100018E
:10028000C051C11107E18C708C50010B02E08C92BF
:1002900001D08C821200B7DF400EE66E650EE66E6E
:1002A000000EE66EB0EC05F0E552E552E5520008AE
:1002B00001E38BD00001606B00016551FF0A72E021
:1002C000EF0A5DE0150A56E0010A41E0070A38E04E
:1002D000010A2FE0030A18E0070A16E0700A01E09D
:1002E00073D0B0DE0001040E606F04010CBFFDD7B7
:1002F000400EE66E650EE66E000EE66E76EC05F0DC
:10030000E552E552E55261D08C848C86A3DE050E61
:100310000001602704010CBFFDD7400EE66E650E9C
:10032000E66E000EE66E76EC05F0E552E552E5521B
:100330004CD08C948C86B3DE0001010E606F45D0EA
:100340008C848C96DBDE0001010E606F3ED0FDDEFA
:10035000050E0001602704010CBFFDD7400EE66EBC
:10036000650EE66E000EE66E76EC05F0E552E5529F
:10037000E5522BD0FFDE0001010E606F26D03CDF7E
:100380000001060E606F04010CBFFDD7400EE66E43
:10039000650EE66E000EE66E76EC05F0E552E5526F
:1003A000E55213D00DEC06F00001636B646B0001A5
:1003B0006307000E645B00016351641103E00000F9
:1003C0000000F5D7FF0001D000D012000401105149
:1003D000600BE842E842E842E842E842000901E0F6
:1003E00055D01151070A51E00B0A4FE0070A40E0CF
:1003F000010A2CE00B0A28E0020A26E0030A22E0A8
:10040000080A12E0010A0EE00F0A0AE0030A01E0FE
:100410003CD00001010EB06F0001040EB76F36D062
:1004200036D834D090D832D00001010EB06F000120
:10043000B90EB16F000EB26F0001B8930001010E4A
:10044000B56F24D0A8D822D0F5D820D00001010E55
:10045000B06F040114510001B16FB26BBA0EB12735
:10046000000EB2230001B8930001010EB56F0ED04B
:100470000001010EB06F04011451EA6ABA0FE96E6F
:10048000000EEA2212C4EFFF01D000D01200800E4D
:100490000401105D57E11351030A34E0010A10E032
:1004A000030A01E04DD00001010EB06F0001540EAF
:1004B000B16F0D0EB26F120E0001B56FB66B40D06A
:1004C0000001010EB06F04011251F66EF76AD89068
:1004D000F636F736EC0EF6260D0EF7220900F5CFAC
:1004E000B1F00A00F5CFB2F0020E0001F76AB125B3
:1004F000F66EB251F7220900F5CFB5F00A00F5CF3C
:10050000B6F01ED00001010EB06F04011251F66E5C
:10051000F76AD890F636F736EE0EF6260D0EF7226D
:100520000900F5CFB1F00A00F5CFB2F0B1C0F6FF87
:10053000B2C0F7FF0800F5500001B56FB66B00D0F0
:100540000001B88312000001010EB06F0F0EE66EBD
:10055000710EE66E0F0EE66E95EC06F0E552E55272
:10056000E552010EE66EBA0EE66E000EE66E95ECF2
:1005700006F0E552E552E55212C4B9F004011251F9
:1005800004E10001050EB76F05D00001060EB76F3C
:1005900061EC05F012000401186B196B0401105195
:1005A0001F0B020A15E0030A0FE0010A01E034D034
:1005B0000001010EB06F02D0040118810001B8A142
:1005C00002D00401188328D00001010EB06F24D09E
:1005D0000001010EB06F040114510F0B080DF35010
:1005E000016A000F006E040E01221451800B01E01D
:1005F000010E040DF35000010024B36F000E012022
:10060000B46FB3C0E9FFB4C0EAFFEF50040B03E0DE
:100610000401010E186F00D00001B0050AE10001CD
:10062000180EB16F040EB26F0001B8930001020EF4
:10063000B56F12000401120510E110511F0B0009E3
:100640000CE10001010EB06F030E0401115D03E126
:100650000001B88102D00001B891040112513AE1C1
:1006600010511F0B020836E114510F0B000932E044
:100670000001010EB06F040114510F0B080DF3506F
:10068000016A000F006E040E01221451800B01E07C
:10069000010E040DF35000010024B36F000E012081
:1006A000B46F030E0401115D07E1840EB3C0E9FFCE
:1006B000B4C0EAFFEF6E0ED014AF06D0B3C0E9FFAE
:1006C000B4C0EAFFEF6A06D0880EB3C0E9FFB4C039
:1006D000EAFFEF6E12006C500BE1040100513C0B7D
:1006E000E842E8420D0802E108D801D03CD804D025
:1006F000040E6C5C01E147D81200D9CFE6FFE1CFD0
:10070000D9FFE6520001AF6BB06BB56BB66BE6EC90
:1007100001F0DF6ADF50006E016A010E005C000E1E
:1007200001581BE20001B05101E017D0F76ADF3435
:10073000FE0BF736F66EF60EF6260D0EF7220900C2
:10074000F5CF00F00800F5CF01F004D001C0FAFFAA
:100750000050F96EFBDFDF2ADDD7DDD8E552E55228
:10076000E7CFD9FF1200020E0001AF5D0AE196D873
:10077000040100BD03D0C80E006F02D0880E006FC8
:1007800001D00FD91200040E0001B75D0AE112C4B6
:100790006EFF6E50000803E2050EB76F02D0030E25
:1007A000B76F0001AF050AE10BD8040104BD03D007
:1007B000C80E046F02D0880E046F01D0F2D8120068
:1007C000D9CFE6FFE1CFD9FF020EE1260001080EE6
:1007D000B55D000EB65905E2B5C0DEFFB6C0DDFF5F
:1007E00003D0080EDE6EDD6A040104930491010E4D
:1007F000DB500413DFCF05F4000EDB500001B55FC2
:10080000010EDB50B65B180EB36F040EB46F00011F
:10081000B8A31ED0D9CFE9FFDACFEAFFEE50ED1032
:1008200016E0B1C0F6FFB2C0F7FF0800F550B3C044
:10083000E9FFB4C0EAFFEF6E0001B32B000EB42352
:10084000B12BB223DF06010E01E2DB06E3D71CD099
:10085000D9CFE9FFDACFEAFFEE50ED1015E0B1C0D5
:10086000E9FFB2C0EAFFEF50B3C0E9FFB4C0EAFF4E
:10087000EF6E0001B32B000EB423B12BB223DF06C1
:10088000010E01E2DB06E4D7020EE15C02E2E16A5E
:10089000E552E16EE552E7CFD9FF1200D9CFE6FF6E
:1008A000E1CFD9FF020EE126030E04010015E76E29
:1008B000010EE7CFDBFF01C4DFFFDE500001B527EB
:1008C000DD50B623180EB16F040EB26FD9CFE9FF19
:1008D000DACFEAFFEE50ED1014E0B1C0E9FFB2C08C
:1008E000EAFFEF50B3C0E9FFB4C0EAFFEF6EB32BED
:1008F000000EB423B12BB223DF06010E01E2DB06AA
:10090000E5D7020EE15C02E2E16AE552E16EE552F2
:10091000E7CFD9FF12006D980001B0510CE104013E
:10092000080E016F100E026F040E036F840E006F2D
:100930000401046F35D0040110AF22D00001B5517D
:100940000401165D0001B6510401175904E216C4F2
:10095000B5F017C4B6F034DF0001010EAF6F04012B
:10096000080E016F100E026F040E036F800E006FF1
:100970000401180E066F040E076FC80E046F10D026
:100980000001020EAF6F0401056BC80E046F040175
:10099000080E016F180E026F040E036FC80E006F71
:1009A00012000001AF6B0401080E016F100E026F00
:1009B000040E036F880E006F0401046B1200040123
:1009C00010511F0B010801E079D0145101E076D0DD
:1009D000060E115D2EE11351230A28E0010A13E0EF
:1009E000030A01E024D00001020EB06F0001B90536
:1009F00005E10001780EB16F0D0EB26F090E000116
:100A0000B56FB66B14D00001020EB06F0001B905CE
:100A100005E10001CF0EB16F0D0EB26F0001B905F7
:100A200004E11D0E0001B56FB66B01D000D00001CE
:100A3000B88304011051600BE842E842E842E84202
:100A4000E842010801E03AD011510B0A31E0080AEE
:100A500021E0090A19E0080A09E00B0A05E0080A82
:100A600001E02CD02CD82AD02BD828D00001020E9F
:100A7000B06F0001BB0EB16F000EB26F0001B893F2
:100A80000001010EB56F1AD00001020EB06F13C441
:100A9000BBF014D00001020EB06F0001BC0EB16FAC
:100AA000000EB26F0001B8930001010EB56F06D0C1
:100AB0000001020EB06F12C4BCF000D01200120090
:100AC00012000001BD6B1E0E716E0401400E096F15
:100AD000200E0A6F040E0B6F880E086F0401600E63
:100AE0000E6F040E0F6F400E0C6F1200D9CFE6FF91
:100AF000E1CFD9FFE652FC0EDB50400805E2400E84
:100B0000F36EFC0EF3CFDBFFDF6AFC0EDB50DF5C25
:100B100019E2DF50E76EFD0EDBCFE9FFFE0EDBCF03
:100B2000EAFFE750E926000EEA22EF50E66EDF50BA
:100B3000EA6A600FE96E040EEA22E552E750EF6EB2
:100B4000DF2AE3D7FC0EDBCF0DF4400E04010C17B7
:100B50000C7D880E0C13E552E552E7CFD9FF120049
:100B6000D9CFE6FFE1CFD9FF0001BD6B040108BF7B
:100B700030D0FC0EDBCF00F00951D880005403E2E6
:100B8000FC0E09C4DBFF0001BD6BFC0EDB50BD5D3C
:100B900019E2BD51EA6A200FE96E040EEA22EF5015
:100BA000E66EBD51E76EFD0EDBCFE9FFFE0EDBCF3B
:100BB000EAFFE750E926000EEA22E552E750EF6E21
:100BC000BD2BE3D70401400E096F0817087D880E7E
:100BD00008130001BD5100D0E552E7CFD9FF120044
:100BE0006DA60FD802D06DB613D80001B70508E185
:100BF0006DBA06D0686A696A69806988020EB76F43
:100C000012006D6A696A6D860001010EB76F1200ED
:100C10006D6A696A0001B76B120008EF06F0000107
:100C2000B75101E13AD06850040B04E06950040B5D
:100C300001E038D86DB231D06850010B04E0695042
:100C4000010B01E050D86850100B04E06950100B04
:100C500001E024D86850400B04E06950400B01E0EB
:100C600037D86850200B04E06950200B01E032D8DF
:100C70006850020B04E06950020B01E032D8030E09
:100C80000001B75D01E209D06850080B06E0695029
:100C9000080B03E06BEC03F0689612006984689817
:100CA0006D8212006D926994689412000001B8A1DF
:100CB0000ED0F8DF6D840001080EBE6F070EBF6F07
:100CC000BE07000EBF5BBE51BF11FAE16D9412006A
:100CD000689C120070A003D0D1EC04F07090689A68
:100CE0001200689212006A6A686A9F0E6B6E7B0E31
:100CF000696E6E6A0F0EE66E710EE66E0F0EE66E90
:100D000014D8E552E552E552160E706E68A602D070
:100D10006896FCD76D98D1EC04F00001B891000101
:100D2000B96B0001030EB76F1200D9CFE6FFE1CF18
:100D3000D9FFFD0EDBCFE9FFFE0EDBCFEAFFFC0E95
:100D4000DB5004E0EE6AFC0EDB06F9D7E552E7CF94
:100D5000D9FF12001201000200000008C0165F0651
:100D600001000102030109022900010102800009BA
:100D70000400000203000000092101000001221DFF
:100D8000000705810340000107050103400001043D
:100D90000309040A034B00310058004D00120353AD
:100DA000004F0032005200200042006F0078001215
:100DB000034600690072006D0077006100720065F3
:100DC000002000550070006400610074006500069A
:100DD00000FF0901A10119012940150026FF007536
:100DE0000895408102190129409102C0660D8F0DBE
:100DF000930D9D0DAF0DBE092A0EF66E000EF76E17
:100E0000000EF86E00010900F550AA6F0900F550B8
:100E1000AB6F03E1AA6701D03DD00900F550A56F83
:100E20000900F550A66F0900F550A76F09000900E9
:100E3000F550E96E0900F550EA6E09000900090055
:100E4000F550A86F0900F550A96F09000900F6CF09
:100E5000ACF0F7CFADF0F8CFAEF0A5C0F6FFA6C06E
:100E6000F7FFA7C0F8FF0001A85302E1A95307E06C
:100E70000900F550EE6EA807F8E2A907F9D7ACC053
:100E8000F6FFADC0F7FFAEC0F8FF0001AA07000EE5
:100E9000AB5BBFD71200938A818AF19E81AA16D0DC
:100EA000A968A69EA69CA680210EA85C02E000EF81
:100EB00010F0A968A86AA69EA69CA684550EA76EE7
:100EC000AA0EA76EA682A6B2FED7A69405D812D8FF
:100ED0004BEC01F0FCD71200F00E8C1695168C84AA
:100EE0008C86140E6F6E0001B76B0001B86B0001A9
:100EF000B96B1200F0EC05F06FBE02D00FEC06F0FB
:100F0000120013EE00F023EE00F0F86A059CFCECF2
:100F100006F096EC07F04BEC07F0FBD7120000EE62
:100F200000F00F0EEE6AEA62FDD712001200000018
:100F3000FFFFFFFFFFFFFFFFFFFFFFFFFFFFFFFFC1
:100F4000FFFFFFFFFFFFFFFFFFFFFFFFFFFFFFFFB1
:100F5000FFFFFFFFFFFFFFFFFFFFFFFFFFFFFFFFA1
:100F6000FFFFFFFFFFFFFFFFFFFFFFFFFFFFFFFF91
:10200000D3EF29F0120000009FEF28F0120000002B
:102010000000000000000000F8EF28F012000000AF
:102020000000000000000000000000008150020BD2
:1020300005E100016151040B01E061818150040B55
:1020400005E100016151080B01E06183120075C0D8
:102050008EF000018E5102E177C08EF076518E270E
:10206000020E8E5D02E2020E8E6F8E51630802E256
:10207000630E8E6F69818EC074F08E51F66EF76AB2
:10208000D890F636F736690EF6264F0EF72209007D
:10209000F5CF7AF00A00F5CF7BF07B510001D30336
:1020A000F3CF7CF0F4CF7DF000017A510001D3032F
:1020B000F3CF8FF0F45000017C27FF0E0001D30313
:1020C000F3CF91F000017B519103F3CF7EF0F4CF79
:1020D0007FF07A519103F3CF90F0F4507E277DAFDB
:1020E0000DD07C697D697A517A257E6F7B517B2189
:1020F0007F6F7C517E5F7D517F5B2BD07FAF0DD09A
:102100007E697F697A517A257C6F7B517B217D6F57
:102110007E517C5F7F517D5B12D07C517C277D514D
:102120007D238FAF03D07C2B000E7D237E517E2735
:102130007F517F2390AF03D07E2B000E7F237C6DD9
:102140007D1F000E7D237E6D7F1F7F237A6D7B1F99
:102150007B231200D9CFE6FFE1CFD9FFFE0EDBCF04
:1021600075F075DFE552E7CFD9FF1200D9CFE6FF52
:10217000E1CFD9FFFE0EDBCF77F0000173A704D0CB
:10218000DBCF75F064DF01D06A81E552E7CFD9FF7C
:1021900012000001836B846B856B866B050ED56E18
:1021A000F294F28A766B876B886B896B8A6B8B6B88
:1021B0008C6B626B636B646B656B666B676B686B78
:1021C000696B6B6B736B73878D6B6C6B6E6B6D6B0D
:1021D000816B00019551F76A310FF66E500EF722B0
:1021E0000800F5CF6FF09551F76A350FF66E500E77
:1021F000F7220800F5CF70F09551F76A390FF66EA7
:10220000500EF7220800F5CF71F09551F76A3D0F97
:10221000F66E500EF7220800F5CF72F0F090F092B3
:10222000F19AF198F086F0880001606B616B6C6B3D
:102230001200F0A003D00001608302D0000160937F
:10224000766B876B886B896B8A6B01DF00016C5141
:1022500062E10001D45123E0F0A005D000016087C5
:10226000616B618704D000016097616B618500013B
:10227000D2AF05D00001715180127251811200015C
:10228000450E786F796979C0D7FF78C0D6FFD58EB3
:10229000010E6C6FD4C080F0020E6E6F38D000015A
:1022A000D2AF05D000017151801272518112F0A09D
:1022B0000FD00001616B618760810001D2A704D05B
:1022C0000001060E806F03D00001020E806F0ED059
:1022D0000001616B618560910001D2A704D000010B
:1022E000020E806F03D00001060E806F020E6C6F2D
:1022F000010E6D6F7CC078F07DC079F079C0D7FF9A
:1023000078C0D6FFD58E6F518012705181126781CF
:10231000F090F092F3D0030E6C5D3DE1EB0E801671
:102320006F0E8116D59EF294836B846B856B866BE2
:10233000606BF0A00ED0616B618760810001D2A755
:1023400004D00001060E806F03D00001020E806FE2
:102350000DD0616B618560910001D2A704D00001AE
:10236000020E806F03D00001060E806F020E6C6FAC
:10237000010E6D6F7CC078F07DC079F079C0D7FF19
:1023800078C0D6FFD58E6F5180127051811267814F
:10239000F090F092B3D0040E6C5D32E1F0A00ED05C
:1023A000616B618760810001D2A704D00001060E35
:1023B000806F03D00001020E806F0DD0616B6185CC
:1023C00060910001D2A704D00001020E806F03D0FB
:1023D0000001060E806F020E6C6F010E6D6F7CC0E7
:1023E00078F07DC079F079C0D7FF78C0D6FFD58E60
:1023F0006F518012705181126781F090F0927ED0FF
:10240000050E6C5D3CE1EB0E80166F0E8116D59EBD
:10241000F29473936B81606BF0A00ED0616B618757
:1024200060810001D2A704D00001060E806F03D0A6
:102430000001020E806F0DD0616B6185609100011B
:10244000D2A704D00001020E806F03D00001060E57
:10245000806F020E6C6F010E6D6F7CC078F07DC0D6
:1024600079F079C0D7FF78C0D6FFD58E6F51801232
:10247000705181126B816781F090F0923FD0060E0F
:102480006C5D32E1F0A00ED0616B6187608100016C
:10249000D2A704D00001060E806F03D00001020E07
:1024A000806F0DD0616B618560910001D2A704D06F
:1024B0000001020E806F03D00001060E806F020E35
:1024C0006C6F010E6D6F7CC078F07DC079F079C0C3
:1024D000D7FF78C0D6FFD58E6F5180127051811210
:1024E0006781F090F0920AD0050E6C5D05E1020E56
:1024F0006E6FF090F09202D0F090F0921200000116
:1025000084514EE089A103D087C076F0A0DD88C059
:1025100087F08AC089F086C085F0F00E0001845DE6
:102520001FE37AC078F07BC079F079C0D7FF78C01C
:10253000D6FFD58E030E6C6F6D6FF00E845D0BE1D0
:102540000001D2A904D00001080E806F03D0000161
:10255000060E806F03D00F0E8415806F64811BD030
:102560006F518012705181127CC078F07DC079F07B
:1025700079C0D7FF78C0D6FFD58E030E6C6F010EE1
:102580006D6F84A103D0060E806F02D0020E806FA3
:1025900084417F0B836F846B866B6381010E02D055
:1025A000000E00D01200D59EF2940001800705E0D5
:1025B00079C0D7FF78C0D6FFD58E6C51040A01E1EF
:1025C00063D2040A01E160D2060A01E14FD2030A94
:1025D00001E126D2060A01E1B3D1010A01E188D066
:1025E000030A23E0060A01E050D280511EE1D70E13
:1025F0008016B70E81166C6B0001D45116E00001F5
:10260000D2AF05D0000171518012725181120001C8
:10261000450E786F796979C0D7FF78C0D6FFD58E1F
:10262000010E6C6FD4C080F030D2000180515FE1A8
:10263000020E6E5D2FE160A70ED0616B6187608135
:102640000001D2A704D00001060E806F03D0000164
:10265000020E806F0DD0616B618560910001D2A781
:1026600004D00001020E806F03D00001060E806FBF
:10267000020E6C6F010E6D6F7CC078F07DC079F03A
:1026800079C0D7FF78C0D6FFD58E6F5180127051B8
:102690008112FBD1030E6E5D0AE131DF000906E114
:1026A000D70E8016B70E811600016C6BEED1050EA9
:1026B0006E5D12E16F51801270518112460E786F7B
:1026C000240E796F79C0D7FF78C0D6FFD58E050E5E
:1026D0006C6F640E806FD9D181A103D0040E6C6F32
:1026E000D4D1D70E8016B70E81166C6BCED1CDD15A
:1026F0006D0528E1805125E1EB0E80166F0E8116E5
:102700007EC078F07FC079F079C0D7FF78C0D6FF5F
:10271000D58E8CDC0001020E6D6F806F7451140831
:1027200006E30001D251400B02E100016185000186
:102730007451270806E30001D251400B02E1000169
:102740006187A3D1020E6D5D01E0FAD0805101E0F6
:10275000E3D00001D2AB0BD08150020B08E08150D6
:10276000040B05E000016051040B01E0616B000106
:10277000618561875BDC000161A18DD061A36AD0B6
:1027800060850001D251070B030A54E0010A43E0BF
:10279000030A22E0010A01E05CD0000160A10ED032
:1027A000616B618560910001D2A704D00001020E27
:1027B000806F03D00001060E806F0DD0616B6187C2
:1027C00060810001D2A704D00001060E806F03D003
:1027D0000001020E806F3DD0000160A30ED0616B3E
:1027E000618760810001D2A704D00001060E806FCE
:1027F00003D00001020E806F0DD0616B6185609186
:102800000001D2A704D00001020E806F03D00001A6
:10281000060E806F1ED00001616B61876081000130
:10282000D2A704D00001060E806F03D00001020E73
:10283000806F0FD00001616B618560910001D2A7AC
:1028400004D00001020E806F03D00001060E806FDD
:1028500000D00ED06095616B618760810001D2A7C6
:1028600004D00001060E806F03D00001020E806FBD
:102870000001020E6C6F010E6D6F7CC078F07DC0A0
:1028800079F079C0D7FF78C0D6FFD58E6F5180120E
:102890007051811240D061A320D06095616B618539
:1028A00060910001D2A704D00001020E806F03D016
:1028B0000001060E806F020E6C6F010E6D6F7CC002
:1028C00078F07DC079F079C0D7FF78C0D6FFD58E7B
:1028D0006F518012705181121ED060950001D55148
:1028E0000EE00001450E786F796979C0D7FF78C096
:1028F000D6FFD58E060E6C6FD5C080F00CD00001CF
:10290000658181A103D0040E6C6F05D0D70E8016AF
:10291000B70E81166C6B13D07451290806E30001C1
:10292000D251400B02E100016185000174512B0876
:1029300006E30001D251400B02E100016187A5D0FE
:1029400080516DE16D0511E1EB0E80166F0E811661
:102950007EC078F07FC079F079C0D7FF78C0D6FF0D
:10296000D58E020E6D6F806F90D0020E6D5D2AE1E4
:10297000830519E06F518012705181127CC078F08C
:102980007DC079F079C0D7FF78C0D6FFD58E010E13
:102990006D6F83A103D0060E806F02D0020E806F90
:1029A000839183430ED07AC078F07BC079F079C0F0
:1029B000D7FF78C0D6FFD58E040E806F030E6D6FE3
:1029C000648163D0030E6D5D2AE199DD000927E182
:1029D0000001766B876B886B896B8A6B27EC10F034
:1029E000000165810001D5510EE00001450E786FB0
:1029F000796979C0D7FF78C0D6FFD58E060E6C6F87
:102A0000D5C080F00CD00001658181A103D0040EF7
:102A10006C6F05D0D70E8016B70E81166C6B35D053
:102A2000805123E1EB0E80166F0E811673936B813C
:102A30000001D5510EE00001450E786F796979C02B
:102A4000D7FF78C0D6FFD58E060E6C6FD5C080F04C
:102A50000CD00001658181A103D0040E6C6F05D0FC
:102A6000D70E8016B70E81166C6B0FD080510BE11C
:102A7000658181A103D0040E6C6F05D0D70E80163E
:102A8000B70E81166C6B01D000D0120016EF10F05B
:102A9000D9CFE6FFE1CFD9FF200EF36EFE0EDBCFDC
:102AA000F4FFF350F45C01E27CD0FE0EDB506008D2
:102AB00001E277D00001845103E0020E8B6F70D0E9
:102AC000FE0EDB50E00FF76A280FF66E4F0EF7226E
:102AD0000800F5CF84F0845103E1010E8B6F60D0C4
:102AE000F29E020E6C5D0DE000019251020B09E1B5
:102AF00000016C0503E0070E6C5D07E1020E6E5DE0
:102B000004E10001846B828348D0FE0EDBCF86F0A7
:102B10006C511BE10001D45118E00001D2AF05D087
:102B2000000171518012725181120001450E786FBF
:102B3000796979C0D7FF78C0D6FFD58E010E6C6F4A
:102B4000D4C080F0030E6E6F28D000016C0503E046
:102B5000070E6C5D07E1050E6E5D01E16B81030EF2
:102B60006E6F1BD073A302D073936B816C5108E11D
:102B70000001D2AF05D00001715180127251811253
:102B800000016C5109E0040E6C5D06E0050E6C5D01
:102B900003E0060E6C5D01E1B2DCF28E00018B6B8E
:102BA00003D00001010E8B6FE552E7CFD9FF120071
:102BB000D9CFE6FFE1CFD9FFE652F29E0001845162
:102BC00003E1030E8C6F2DD0200EF36EFE0EDBCFD3
:102BD000F4FFF350F45C1BE3FE0EDB50600817E3D8
:102BE000FE0EDB50E00FF76A280FF66E4F0EF7224D
:102BF0000800F550DF6EDF5003E1010E8C6F06D048
:102C0000DFCF84F0FE0EDBCF86F08C6B0AD0FE0E99
:102C1000DB5005E1846B866B8C6B668102D0010E04
:102C20008C6FF28EE552E552E7CFD9FF1200D9CF73
:102C3000E6FFE1CFD9FFE652FE0EDB50DF6EF29EDB
:102C4000D9CFE9FFDACFEAFFEF50020B51E00001E4
:102C50006C51070A48E0030A34E0020A32E0060A2F
:102C600001E046D073830001D45118E00001D2AFD7
:102C700005D0000171518012725181120001450E80
:102C8000786F796979C0D7FF78C0D6FFD58E010EED
:102C90006C6FD4C080F0050E6E6F12D000016F51C2
:102CA000801270518112460E786F240E796F79C0B0
:102CB000D7FF78C0D6FFD58E050E6C6F640E806F7F
:102CC00017D06F51801270518112460E786F240E0A
:102CD000796F79C0D7FF78C0D6FFD58E050E6C6F9F
:102CE000640E806F05D06E5102E1050E6E6F00D04C
:102CF000D9CFE9FFDACFEAFFEF50010B3CE0050E38
:102D000000016C5D25E1EB0E80166F0E8116D59EDD
:102D1000F29473930001D5510EE00001450E786FD7
:102D2000796979C0D7FF78C0D6FFD58E060E6C6F53
:102D3000D5C080F00CD00001658181A103D0040EC4
:102D40006C6F05D0D70E8016B70E81166C6B13D042
:102D50006C0511E1050E6E5D0EE17393D59EF29444
:102D6000658181A103D0040E6C6F05D0D70E80164B
:102D7000B70E81166C6BD9CFE9FFDACFEAFFEF50BF
:102D8000080B02E000017387D9CFE9FFDACFEAFF31
:102D9000EF50040B02E000017397F28EE552E5520A
:102DA000E7CFD9FF1200D9CFE6FFE1CFD9FFF29EDE
:102DB0000001845105E0FE0EDBCF88F08A8104D04B
:102DC000FE0EDBCF87F08981F28E00D0E552E7CF8F
:102DD000D9FF1200F29E030E00016C5D03E0050EA8
:102DE0006C5D2DE1EB0E80166F0E8116D59EF29470
:102DF000766B876B886B896B8A6B27EC10F0000110
:102E000065810001D5510EE00001450E786F7969AA
:102E100079C0D7FF78C0D6FFD58E060E6C6FD5C0AF
:102E200080F00CD00001658181A103D0040E6C6F8D
:102E300005D0D70E8016B70E81166C6B13D06C05BB
:102E400011E1020E6E5D0EE0D59EF2946581658102
:102E500081A103D0040E6C6F05D0D70E8016B70E7B
:102E600081166C6B836B846B856B866B7393F28EB0
:102E7000120000016C5137E0060E6C5D03E1070E95
:102E80006C6F31D0EB0E80166F0E8116D59EF294CA
:102E9000050E6C5D02E173936B81030E6C5D0FE1B7
:102EA00082856581766B876B886B896B8A6B27EC73
:102EB00010F000016581836B846B856B866B450E1A
:102EC000786F796979C0D7FF78C0D6FFD58E070EA5
:102ED0006C6F6E6B0001D55103E0D5C080F003D05C
:102EE0000001050E806F00019551F76A310FF66EF3
:102EF000500EF7220800F5CF6FF09551F76A350FA5
:102F0000F66E500EF7220800F5CF70F09551F76A73
:102F1000390FF66E500EF7220800F5CF71F095517B
:102F2000F76A3D0FF66E500EF7220800F5CF72F0EB
:102F30001200F29E00017151801272518112818142
:102F40006C511EE10001D45118E00001D2AF05D050
:102F5000000171518012725181120001450E786F8B
:102F6000796979C0D7FF78C0D6FFD58E010E6C6F16
:102F7000D4C080F0040E6E6F03D00001040E6C6F9D
:102F8000F28E1200F29E0001816B040E6C5D05E171
:102F9000D70E8016B70E81166C6BF28E1200D9CF49
:102FA000E6FFE1CFD9FFE652FE0EDB50DF6ED9CF50
:102FB000E9FFDACFEAFFEF50070B030804E3DFCFA6
:102FC000D2F00001CC89E552E552E7CFD9FF1200DB
:102FD000D9CFE6FFE1CFD9FFF29EFE0EDBCFD3F0D3
:102FE0000001CC8B27EC10F0F28EE552E7CFD9FF31
:102FF0001200D9CFE6FFE1CFD9FFFE0EDBCFD4F030
:103000000001CC8DE552E7CFD9FF1200D9CFE6FF02
:10301000E1CFD9FFFE0EDBCFD5F00001CC8FE5521A
:10302000E7CFD9FF120075C08DF000018D5100D09F
:1030300012000001D35100D012000001775100D0DE
:103040001200D9CFE6FFE1CFD9FFE652DF6A0001D7
:103050006C51010A16E0040A10E0060A0AE0010AAF
:1030600004E0DF90DF92DF9424D0DF80DF92DF94F2
:1030700020D0DF90DF82DF941CD0DF80DF82DF94FE
:1030800018D06E51050A10E0060A0AE0010A04E0B1
:10309000DF90DF92DF940CD0DF80DF92DF9408D0E6
:1030A000DF90DF82DF9404D0DF80DF82DF9400D006
:1030B00000D0845101E1DF88000192B3DF86DF5048
:1030C00000D0E552E552E7CFD9FF120000018B5145
:1030D00000D0120000018C5100D012000001765186
:1030E00000D01200D9CFE6FFE1CFD9FFE65273C07E
:1030F000DFFFD9CFE9FFDACFEAFFEF50020B01E1A2
:10310000DF80D9CFE9FFDACFEAFFEF50080B01E10A
:10311000DF84DF5000D0E552E552E7CFD9FF12003F
:10312000000169A106D0696B75518D5D02E0010E49
:1031300002D0000E00D0120000016AA103D06A6B19
:10314000010E02D0000E00D0120000016BA103D0CE
:103150006B6B010E02D0000E00D01200000163A1C3
:1031600003D0636B010E02D0000E00D012000001EC
:1031700066A103D0666B010E02D0000E00D01200D3
:10318000000164A103D0646B010E02D0000E00D0D8
:103190001200000165A103D0656B010E02D0000E84
:1031A00000D01200000167A103D0676B010E02D0AE
:1031B000000E00D01200D9CFE6FFE1CFD9FFE652D2
:1031C000F29E82C0DFFF0001826BF28EDF5000D0E2
:1031D000E552E552E7CFD9FF12000001855100D03A
:1031E0001200806A0E0EC16EC10E926E816A070EC9
:1031F000936E826A946A966A846A836AF00E956E08
:10320000848E8C908C948C928C96FEEC20F01AEC30
:103210001FF021EC28F0C9EC10F03DEF27F09FECF7
:103220001FF0A4EC21F0060E0001ED5D03E36D50EC
:10323000020B01E002D021D82BDB1200D9CFE6FF30
:10324000E1CFD9FF04010CAF03D066EC26F0FAD72A
:10325000FE0EDBCFB9F0FD0EDBCFBAF0020EE66E4C
:10326000B90EE66E000EE66ECFEC25F0E552E552A3
:10327000E552E552E7CFD9FF1200020EE66EC10E0D
:10328000E66E000EE66E09EC26F0E552E552E552D8
:103290000001B86F020E0001B85D01E0F8D2000134
:1032A000C151350A01E1DDD2010A01E1CCD2070AA0
:1032B00001E1BCD2010A01E1B0D2030A01E1A0D2CE
:1032C000010A01E18FD2130A01E17ED2010A01E174
:1032D0006DD2030A01E15CD2010A01E14BD23D0A41
:1032E00001E13FD2010A01E133D2070A01E122D212
:1032F000010A01E112D2030A01E102D2010A01E14D
:10330000F1D10F0A01E1E7D1010A01E1D6D1030AA7
:1033100001E1C9D1010A01E1B8D1070A01E1A7D150
:10332000010A01E197D1030A01E184D1010A01E117
:1033300078D1180A01E156D10A0A01E14CD1030AF9
:1033400001E142D1010A01E09AD20001C251350ADD
:1033500001E128D1010A01E11CD1070A01E111D1E3
:10336000010A01E105D1030A01E1FAD0010A01E1F4
:10337000EED0130A01E1E2D0010A01E1D6D0030A3E
:1033800001E1CAD0010A01E1BED03D0A01E1B2D09B
:10339000010A01E1A6D0070A01E19AD0010A01E180
:1033A0008FD0030A01E184D0010A01E178D00F0A2D
:1033B0006FE0010A64E0030A5BE0010A50E0070ADB
:1033C00045E0010A3BE0030A30E0010A25E0180A63
:1033D0001CE00A0A13E0030A0AE0010A01E0EBD04C
:1033E000100EE66EE66A2ADFE552E552ECD0E66A98
:1033F000010EE66E23DFE552E552E5D0E66A020EE5
:10340000E66E1CDFE552E552DED0E66A080EE66E97
:1034100015DFE552E552D7D021EC18F0E66E100E1C
:10342000E66E0CDFE552E552CED013EC18F0E66EF6
:10343000110EE66E03DFE552E552C5D0D2C0E6FFBD
:10344000120EE66EFBDEE552E552BDD066EC18F0DA
:10345000E66E130EE66EF2DEE552E552B4D06AEC8B
:1034600018F0E66E140EE66EE9DEE552E552ABD0DA
:10347000E66A150EE66EE2DEE552E552A4D072EC85
:1034800018F0E66E160EE66ED9DEE552E5529BD0D8
:10349000E66A170EE66ED2DEE552E55294D06EEC87
:1034A00018F0E66E180EE66EC9DEE552E5528BD0D6
:1034B000D4C0E6FF190EE66EC1DEE552E55283D0B8
:1034C000D5C0E6FF1A0EE66EB9DEE552E5527BD0B6
:1034D00019EC18F0E66E1B0EE66EB0DEE552E55212
:1034E00072D01DEC18F0E66E1C0EE66EA7DEE552FB
:1034F000E55269D0EDEC18F0E66E1D0EE66E9EDE2C
:10350000E552E55260D084EC27F0E66E200EE66EC0
:1035100095DEE552E55257D088EC27F0E66E210E95
:10352000E66E8CDEE552E5524ED08CEC27F0E66E6E
:10353000220EE66E83DEE552E55245D090EC27F090
:10354000E66E230EE66E7ADEE552E5523CD0EAECFA
:103550001FF0E66E300EE66E71DEE552E55233D0B6
:10356000CEC0E6FF310EE66E69DEE552E5522BD0A5
:10357000EEEC1FF0E66E320EE66E60DEE552E552CE
:1035800022D0CFC0E6FF330EE66E58DEE552E5529C
:103590001AD063EC20F0E66E340EE66E4FDEE55294
:1035A000E55211D08FEC20F0E66E350EE66E46DE69
:1035B000E552E55208D0C2C0E6FF7F0EE66E3EDE61
:1035C000E552E55200D063D1E66A010EE66E36DEC2
:1035D000E552E5525CD1E66A020EE66E2FDEE55258
:1035E000E55255D1210E0001C25D13E140EC22F0FD
:1035F00064EC26F00001C96BCA6B0001C907000E1C
:10360000CA5B0001C951CA1103E000000000F5D7F0
:10361000FF00010EE66E080EE66E10DEE552E55282
:1036200036D121EC18F0E66E100EE66E07DEE5529C
:10363000E5522DD1F29EC2C0E6FFAAEC10F0E55291
:10364000F28E13EC18F0E66E110EE66EF7DDE55221
:10365000E5521DD1C2C0E6FFCFEC17F0E552D2C053
:10366000E6FF120EE66EEADDE552E55210D1C2C069
:10367000E6FF48EC15F0E55266EC18F0E66E130E26
:10368000E66EDCDDE552E55202D1C2C0E6FFD8ECC1
:1036900015F0E5526AEC18F0E66E140EE66ECEDD1B
:1036A000E552E552F4D0EAEC16F0010EE66E150E86
:1036B000E66EC4DDE552E552EAD0C2C0E6FF17EC83
:1036C00016F0E55272EC18F0E66E160EE66EB6DDF8
:1036D000E552E552DCD0E66A170EE66EAFDDE55244
:1036E000E552D5D0C2C0E6FFD3EC16F0E5526EEC41
:1036F00018F0E66E180EE66EA1DDE552E552C7D071
:10370000C2C0E6FFF9EC17F0E552D4C0E6FF190E8F
:10371000E66E94DDE552E552BAD0C2C0E6FF06EC93
:1037200018F0E552D5C0E6FF1A0EE66E87DDE552C9
:10373000E552ADD0C2C0E6FFE8EC17F0E55219EC57
:1037400018F0E66E1B0EE66E79DDE552E5529FD06D
:103750001DEC18F0E66E1C0EE66E70DDE552E552CB
:1037600096D0EDEC18F0E66E1D0EE66E67DDE552C4
:10377000E5528DD0C2C0E6FF44EC27F0E55284EC60
:1037800027F0E66E200EE66E59DDE552E5527FD059
:10379000C2C0E6FF54EC27F0E55288EC27F0E66E55
:1037A000210EE66E4BDDE552E55271D0C2C0E6FF58
:1037B00064EC27F0E5528CEC27F0E66E220EE66E04
:1037C0003DDDE552E55263D0C2C0E6FF74EC27F060
:1037D000E55290EC27F0E66E230EE66E2FDDE55203
:1037E000E55255D0C2C0E6FFDCEC1FF0E552EAEC32
:1037F0001FF0E66E300EE66E21DDE552E55247D051
:10380000C2C0E6FFAFEC1FF0E552CEC0E6FF310EBE
:10381000E66E14DDE552E5523AD0EEEC1FF0E66EAE
:10382000320EE66E0BDDE552E55231D0C2C0E6FF46
:10383000C1EC1FF0E552CFC0E6FF330EE66EFEDCB2
:10384000E552E55224D0C2C0E6FFFDEC1FF0E55280
:1038500063EC20F0E66E340EE66EF0DCE552E552E5
:1038600016D0C2C0E6FF30EC20F0E5528FEC20F01D
:10387000E66E350EE66EE2DCE552E55208D0C1C0D8
:10388000E6FF7F0EE66EDADCE552E55200D012006C
:1038900004010CBFB0D0A5EC18F0000909E072ECEF
:1038A00018F0E66E160EE66EC9DCE552E552A3D0BE
:1038B000DBEC18F00001CB6FCB5108E0CBC0E6FF8A
:1038C000150EE66EBBDCE552E55295D0B7EC18F06C
:1038D000000908E0030EE66E170EE66EAFDCE55257
:1038E000E55289D0AEEC18F0000909E0EDEC18F0D3
:1038F000E66E1D0EE66EA2DCE552E5527CD0C0EC11
:1039000018F0000908E0010EE66E170EE66E96DC70
:10391000E552E55270D0C9EC18F0000908E0020E3B
:10392000E66E170EE66E8ADCE552E55264D0D2EC04
:1039300018F0000908E0040EE66E170EE66E7EDC55
:10394000E552E55258D090EC18F0000909E013EC6C
:1039500018F0E66E110EE66E71DCE552E5524BD0C2
:103960009CEC18F0000909E01DEC18F0E66E1C0E46
:10397000E66E64DCE552E5523ED0F4EC1FF000093F
:1039800008E0EEEC1FF0E66E320EE66E57DCE55214
:10399000E5520001B4510AE0B4C0E6FF0A0EE66E3B
:1039A0004DDCE552E5520001B46B25D0B5510AE07B
:1039B000B5C0E6FF0B0EE66E41DCE552E5520001B4
:1039C000B56B19D0B6510AE0B6C0E6FF0C0EE66E34
:1039D00035DCE552E5520001B66B0DD0B7510BE076
:1039E000B7C0E6FF0D0EE66E1EEC19F0E552E5528B
:1039F0000001B76B00D01200D9CFE6FFE1CFD9FFAD
:103A00000001080EB36FFE0EDBAE02D08D8201D036
:103A10008D92000000000001B3078D80FE0EDBCF09
:103A2000E7FFE79EE746FE0EE7CFDBFF0000000062
:103A30008D900001B351E7E1E552E7CFD9FF1200C5
:103A40000001A9A507D096C09AF09CC0A4F09DC023
:103A5000A5F02AD0A9A707D097C09AF09EC0A4F0DD
:103A60009FC0A5F021D0A8A310D0A8A507D099C0C9
:103A70009AF0A2C0A4F0A3C0A5F006D097C09AF017
:103A80009EC0A4F09FC0A5F00FD0A8A507D098C0F5
:103A90009AF0A0C0A4F0A1C0A5F006D096C09AF0FC
:103AA0009CC0A4F09DC0A5F0C00EA5139A51040BB4
:103AB00006E00001CE51080B02E00001A5890001DB
:103AC000A651A41902E1A751A5190AE08992A5C03F
:103AD000E6FF92DFE552A4C0E6FF8EDFE552898261
:103AE00000019AA102D08C8001D08C909AA302D0C0
:103AF0008C8201D08C929AC09BF0A4C0A6F0A5C085
:103B0000A7F01200D9CFE6FFE1CFD9FFE65293C06C
:103B1000DFFFF29E0001926BA9A104D09291A8B19F
:103B200092830DD0A9A306D0928194C0DFFFA8A1F3
:103B3000928305D0A8A103D0928194C0DFFF955154
:103B4000DF5C04E0DFCF95F039EC17F0F28E000176
:103B5000CEA90CD0FC0E821600019551F76ADA0F3F
:103B6000F66E530EF7220800F5508212000192A162
:103B700003D08C868C9402D08C848C96E552E552CE
:103B8000E7CFD9FF1200D9CFE6FFE1CFD9FFE65248
:103B9000DF6A0001A951100B06E1A851080B06E0ED
:103BA0009251020B03E199EC17F002D0C2EC17F02E
:103BB000E552E552E7CFD9FF12000001CE51070BC5
:103BC000010A01E1DAD0030A01E183D0020A01E02F
:103BD00030D10001010E966F070E986F020E976F9D
:103BE000070E996F9351F66EF76AD890F636F7364E
:103BF000D20EF626530EF7220900F5CF02F0080088
:103C0000F5CF03F09351F66EF76AD890F636F73693
:103C1000C20EF626530EF7220900F55000010210DD
:103C200000019C6F0900F5500001031000019D6F19
:103C30009451F66EF76AD890F636F736CA0EF62625
:103C4000530EF7220900F5CF02F00800F5CF03F07C
:103C50009351F66EF76AD890F636F736C20EF6260E
:103C6000530EF7220900F550000102100001A06F69
:103C70000900F550000103100001A16F9451F66E88
:103C8000F76AD890F636F736D20EF626530EF7229C
:103C90000900F5CF02F00800F5CF03F09451F66E5D
:103CA000F76AD890F636F736C20EF626530EF7228C
:103CB0000900F5500001021000019E6F0900F55047
:103CC0000001031000019F6FA0C0A2F0A1C0A3F0EB
:103CD000B0D00001050E966F070E986F060E976F15
:103CE000070E996F9351F66EF76AD890F636F7364D
:103CF000C20EF626530EF7220900F5CF9CF00A00FB
:103D0000F5CF9DF09451F66EF76AD890F636F736F7
:103D1000CA0EF626530EF7220900F5CF02F008006E
:103D2000F5CF03F09351F66EF76AD890F636F73672
:103D3000C20EF626530EF7220900F55000010210BC
:103D40000001A06F0900F550000103100001A16FF0
:103D50009451F66EF76AD890F636F736CA0EF62604
:103D6000530EF7220900F5CF9EF00A00F5CF9FF021
:103D7000A0C0A2F0A1C0A3F05CD00001010E966F1C
:103D8000986F020E976F996F9351F66EF76AD890FD
:103D9000F636F736CA0EF626530EF7220900F5CF8F
:103DA00002F00800F5CF03F09351F66EF76AD89051
:103DB000F636F736C20EF626530EF7220900F550F6
:103DC0000001021000019C6F0900F5500001031072
:103DD00000019D6F9CC0A0F09DC0A1F09451F66EB3
:103DE000F76AD890F636F736CA0EF626530EF72243
:103DF0000900F5CF02F00800F5CF03F09451F66EFC
:103E0000F76AD890F636F736C20EF626530EF7222A
:103E10000900F5500001021000019E6F0900F550E5
:103E20000001031000019F6F9EC0A2F09FC0A3F08D
:103E300000D01200E66AE0DDE552E66ADDDDE5521B
:103E40008A8A8982D0C093F0D1C094F093C095F053
:103E50000001A86BAB6BAC6BAD6BA96BAA6BAE6BC7
:103E6000AF6BB06BB16BB26B09D8CFC0E6FF89D82E
:103E7000E552A3DEE5DD46DEC3EF1DF00001AE51E5
:103E800002E0AE070FD083A807D0A9A504D0A9955A
:103E9000AB810A0EAE6F06D0A9B504D0A985AB815F
:103EA0000A0EAE6FAF5102E0AF070FD083AA07D062
:103EB000A9A704D0A997AB810A0EAF6F06D0A9B706
:103EC00004D0A987AB810A0EAF6FB05102E0B007F2
:103ED0000FD083AC07D0A9A104D0A991AC810A0E60
:103EE000B06F06D0A9B104D0A981AC810A0EB06F21
:103EF000B15102E0B1070FD083AE07D0A9A304D01F
:103F0000A993AC810A0EB16F06D0A9B304D0A983DE
:103F1000AC810A0EB16FB25102E0B2070FD081A09E
:103F200007D0A9A904D0A999AD810A0EB26F06D015
:103F3000A9B904D0A989AD810A0EB26F120000019F
:103F4000ABA102D0AB6B7CDD0001ACA102D0AC6BAD
:103F5000D9DD0001ADA102D0AD6B15DE1200D9CFC5
:103F6000E6FFE1CFD9FFFE0EDB501F0B0001CE6F45
:103F70000001CC8122DE64DDC5DDE552E7CFD9FF4B
:103F80001200D9CFE6FFE1CFD9FFFE0EDBCFCFF095
:103F90000001CC878D8000008A9A00008D90110E60
:103FA000E66E2ADDE552CFC0E6FF26DDE5528A8ABD
:103FB000E552E7CFD9FF1200D9CFE6FFE1CFD9FF15
:103FC000FE0EDBCFA8F03CDD9DDDDDDDE552E7CF69
:103FD000D9FF12000001A85100D01200A9C0AAF018
:103FE0000001AA5100D012000001AA51A95D02E00F
:103FF000010E02D0000E00D01200D9CFE6FFE1CFB3
:10400000D9FFE652FE0EDB50DF6ED9CFE9FFDACFE3
:10401000EAFFEF50100B0BE0D9CFE9FFDACFEAFF50
:10402000EF500F0B030B0001D06F0001CC83D9CFF1
:10403000E9FFDACFEAFFEF50200B0DE0F29ED9CF77
:10404000E9FFDACFEAFFEF500F0B0001936F5ADD63
:10405000F28EB3DDF5DCE552E552E7CFD9FF120071
:10406000D9CFE6FFE1CFD9FFE652FE0EDB50DF6E7F
:10407000D9CFE9FFDACFEAFFEF50100B0BE0D9CF31
:10408000E9FFDACFEAFFEF500F0B030B0001D16F0E
:104090000001CC85D9CFE9FFDACFEAFFEF50200B42
:1040A0000DE0F29ED9CFE9FFDACFEAFFEF500F0B18
:1040B0000001946F27DDF28E80DDC2DCE552E5520F
:1040C000E7CFD9FF1200D9CFE6FFE1CFD9FFE65203
:1040D00000019351026ED9CFE9FFDACFEAFF025017
:1040E0000F0BF36EF00EEF14F310EF6E0001D051D2
:1040F000026ED9CFE9FFDACFEAFF02500F0BF36E61
:10410000F346F346F346F3460F0EEF14F310EF6E4B
:10411000DF5000D0E552E552E7CFD9FF1200D9CFEA
:10412000E6FFE1CFD9FFE65200019451026ED9CFEC
:10413000E9FFDACFEAFF02500F0BF36EF00EEF1437
:10414000F310EF6E0001D151026ED9CFE9FFDACF43
:10415000EAFF02500F0BF36EF346F346F346F346C5
:104160000F0EEF14F310EF6EDF5000D0E552E55262
:10417000E7CFD9FF1200D9CFE6FFE1CFD9FFFE0E7E
:10418000DB50A96EA69EA69CA680A85000D0E55242
:10419000E7CFD9FF1200D9CFE6FFE1CFD9FFFE0E5E
:1041A000DB50A96EFD0EDB50A86EA69EA69CA684D1
:1041B000550EA76EAA0EA76EA682A6B2FED7A6942B
:1041C00000D0E552E7CFD9FF1200D9CFE6FFE1CF0B
:1041D000D9FFF29EFE0EDB50A96EFD0EDB50A86EDD
:1041E000A69EA69CA684550EA76EAA0EA76EA682B2
:1041F000F28E00D0E552E7CFD9FF1200D9CFE6FF0B
:10420000E1CFD9FFE6520001CC6BCD6BE66AB3DF9C
:10421000E552010812E1010EE66EADDFE55223081A
:104220000CE1020EE66EA7DFE552450806E1030E3B
:10423000E66EA1DFE552670852E0010EE66EE66A1F
:10424000AADFE552E552230EE66E010EE66EA3DF0D
:10425000E552E552450EE66E020EE66E9CDFE55233
:10426000E552670EE66E030EE66E95DFE552E55207
:10427000E66A040EE66E8FDFE552E552E66A050E49
:10428000E66E89DFE552E552E66AE66884DFE552CC
:10429000E552E66A060EE66E7EDFE552E552800ED6
:1042A000E66E070EE66E77DFE552E552E66A080E27
:1042B000E66E71DFE552E552E66A090EE66E6BDFE7
:1042C000E552E552E66A0A0EE66E65DFE552E55212
:1042D000010EE66E0B0EE66E5EDFE552E552040E51
:1042E000E66E49DFE5520001CE6F050EE66E43DF54
:1042F000E5520001D26F060EE66E3DDFE552000189
:10430000CF6F070EE66E37DFE5520001D36F080E60
:10431000E66E31DFE5520001D46F090EE66E2BDF49
:10432000E5520001D56F0A0EE66E25DFE552000169
:10433000D06F0B0EE66E1FDFE5520001D16FE55224
:10434000E552E7CFD9FF1200A6B299D00001CCA167
:1043500011D0040EE66E0FDFE5520001CE5D07E0DE
:10436000CEC0E6FF040EE66E30DFE552E5520001F6
:10437000CC9185D0CCA911D0050EE66EFCDEE552BD
:104380000001D25D07E0D2C0E6FF050EE66E1DDF3C
:10439000E552E5520001CC9972D0CCA311D00A0E9F
:1043A000E66EE9DEE5520001D05D07E0D0C0E6FF31
:1043B0000A0EE66E0ADFE552E5520001CC935FD0AB
:1043C000CCA511D00B0EE66ED6DEE5520001D15D14
:1043D00007E0D1C0E6FF0B0EE66EF7DEE552E552D0
:1043E0000001CC954CD0CCA711D0060EE66EC3DEF2
:1043F000E5520001CF5D07E0CFC0E6FF060EE66E96
:10440000E4DEE552E5520001CC9739D0CCAB11D0B7
:10441000070EE66EB0DEE5520001D35D07E0D3C0C3
:10442000E6FF070EE66ED1DEE552E5520001CC9BB9
:1044300026D0CCAD11D0080EE66E9DDEE55200010F
:10444000D45D07E0D4C0E6FF080EE66EBEDEE5529E
:10445000E5520001CC9D13D0CCAF11D0090EE66E11
:104460008ADEE5520001D55D07E0D5C0E6FF090E02
:10447000E66EABDEE552E5520001CC9F00D01200A3
:10448000210EE66EE66887DEE552E5521200040171
:104490001051600BE842E842E842E842E842000975
:1044A00001E055D01151070A51E00B0A4FE0070A0D
:1044B00040E0010A2CE00B0A28E0020A26E0030A89
:1044C00022E0080A12E0010A0EE00F0A0AE0030ADD
:1044D00001E03CD00001010EE16F0001040EED6F20
:1044E00036D036D834D090D832D00001010EE16FEA
:1044F0000001EF0EE26F000EE36F0001EE9300018A
:10450000010EE66F24D0A8D822D0EDD820D000012B
:10451000010EE16F040114510001E26FE36BF00E34
:10452000E227000EE3230001EE930001010EE66F87
:104530000ED00001010EE16F04011451EA6AF00F80
:10454000E96E000EEA2212C4EFFF01D000D0120083
:10455000800E0401105D57E11351030A34E0010A93
:1045600010E0030A01E04DD00001010EE16F0001EF
:10457000260EE26F520EE36F120E0001E66FE76B3C
:1045800040D00001010EE16F04011251F66EF76A8E
:10459000D890F636F736C30EF626520EF7220900EB
:1045A000F5CFE2F00A00F5CFE3F0020E0001F76A62
:1045B000E225F66EE351F7220900F5CFE6F00A0096
:1045C000F5CFE7F01ED00001010EE16F040112519A
:1045D000F66EF76AD890F636F736C70EF626520E04
:1045E000F7220900F5CFE2F00A00F5CFE3F0E2C0D0
:1045F000F6FFE3C0F7FF0800F5500001E66FE76B38
:1046000000D00001EE8312000001010EE16F0F0ED9
:10461000E66E710EE66E0F0EE66EF0EC26F0E552D9
:10462000E552E552010EE66EF00EE66E000EE66E05
:10463000F0EC26F0E552E552E55212C4EFF0040129
:10464000125104E10001050EED6F05D00001060EC8
:10465000ED6FBAEC25F012000401186B196B040120
:1046600010511F0B020A0DE0030A07E0010A01E0E6
:104670002CD00001010EE16F28D00001010EE16F86
:1046800024D00001010EE16F040114510F0B080D3D
:10469000F350036A000F026E040E03221451800BC4
:1046A00001E0010E040DF35000010224E46F000E3E
:1046B0000320E56FE4C0E9FFE5C0EAFFEF50040B1B
:1046C00003E00401010E186F00D00001E1050AE1CA
:1046D0000001180EE26F040EE36F0001EE9300017B
:1046E000020EE66F12000401120510E110511F0BBB
:1046F00000090CE10001010EE16F030E0401115DE0
:1047000003E10001EE8102D00001EE91040112519B
:104710003AE110511F0B020836E114510F0B00094A
:1047200032E00001010EE16F040114510F0B080D7E
:10473000F350036A000F026E040E03221451800B23
:1047400001E0010E040DF35000010224E46F000E9D
:104750000320E56F030E0401115D07E1840EE4C040
:10476000E9FFE5C0EAFFEF6E0ED014AF06D0E4C05B
:10477000E9FFE5C0EAFFEF6A06D0880EE4C0E9FF72
:10478000E5C0EAFFEF6E12006C500BE1040100512E
:104790003C0BE842E8420D0802E108D801D03CD8C1
:1047A00004D0040E6C5C01E147D81200D9CFE6FFBB
:1047B000E1CFD9FFE6520001E06BE16BE66BE76BFE
:1047C00047EC22F0DF6ADF50026E036A010E025CE2
:1047D000000E03581BE20001E15101E017D0F76A17
:1047E000DF34FE0BF736F66ECF0EF626520EF722AA
:1047F0000900F5CF02F00800F5CF03F004D003C0A4
:10480000FAFF0250F96EFBDFDF2ADDD7DDD8E55273
:10481000E552E7CFD9FF1200020E0001E05D0AE188
:1048200096D8040100BD03D0C80E006F02D0880ED8
:10483000006F01D00FD91200040E0001ED5D0AE1F6
:1048400012C46EFF6E50000803E2050EED6F02D039
:10485000030EED6F0001E0050AE10BD8040104BD71
:1048600003D0C80E046F02D0880E046F01D0F2D8B6
:104870001200D9CFE6FFE1CFD9FF020EE1260001F9
:10488000080EE65D000EE75905E2E6C0DEFFE7C070
:10489000DDFF03D0080EDE6EDD6A0401049304918F
:1048A000010EDB500413DFCF05F4000EDB500001D6
:1048B000E65F010EDB50E75B180EE46F040EE56F58
:1048C0000001EEA31ED0D9CFE9FFDACFEAFFEE5008
:1048D000ED1016E0E2C0F6FFE3C0F7FF0800F55068
:1048E000E4C0E9FFE5C0EAFFEF6E0001E42B000E33
:1048F000E523E22BE323DF06010E01E2DB06E3D72B
:104900001CD0D9CFE9FFDACFEAFFEE50ED1015E069
:10491000E2C0E9FFE3C0EAFFEF50E4C0E9FFE5C011
:10492000EAFFEF6E0001E42B000EE523E22BE32308
:10493000DF06010E01E2DB06E4D7020EE15C02E2D3
:10494000E16AE552E16EE552E7CFD9FF1200D9CF17
:10495000E6FFE1CFD9FF020EE126030E04010015A8
:10496000E76E010EE7CFDBFF01C4DFFFDE50000181
:10497000E627DD50E723180EE26F040EE36FD9CF70
:10498000E9FFDACFEAFFEE50ED1014E0E2C0E9FFF4
:10499000E3C0EAFFEF50E4C0E9FFE5C0EAFFEF6ED5
:1049A000E42B000EE523E22BE323DF06010E01E2F8
:1049B000DB06E5D7020EE15C02E2E16AE552E16E58
:1049C000E552E7CFD9FF12006D980001E1510CE1EB
:1049D0000401080E016F100E026F040E036F840EA7
:1049E000006F0401046F35D0040110AF22D0000124
:1049F000E6510401165D0001E7510401175904E274
:104A000016C4E6F017C4E7F034DF0001010EE06FD2
:104A10000401080E016F100E026F040E036F800E6A
:104A2000006F0401180E066F040E076FC80E046FA6
:104A300010D00001020EE06F0401056BC80E046F78
:104A40000401080E016F180E026F040E036FC80EEA
:104A5000006F12000001E06B0401080E016F100EE0
:104A6000026F040E036F880E006F0401046B1200C6
:104A7000040110511F0B010801E079D0145101E02D
:104A800076D0060E115D2EE11351230A28E0010AAB
:104A900013E0030A01E024D00001020EE16F0001DF
:104AA000EF0505E100014A0EE26F520EE36F090EB9
:104AB0000001E66FE76B14D00001020EE16F000108
:104AC000EF0505E10001A10EE26F520EE36F000158
:104AD000EF0504E1220E0001E66FE76B01D000D084
:104AE0000001EE8304011051600BE842E842E84205
:104AF000E842E842010801E03AD011510B0A31E0E6
:104B0000080A21E0090A19E0080A09E00B0A05E091
:104B1000080A01E02CD02CD82AD02BD828D00001AC
:104B2000020EE16F0001F40EE26F000EE36F000170
:104B3000EE930001010EE66F1AD00001020EE16F44
:104B400013C4F4F014D00001020EE16F0001F50E61
:104B5000E26F000EE36F0001EE930001010EE66FBD
:104B600006D00001020EE16F12C4F5F000D0120071
:104B7000120012000001F66B1E0E716E0401080E89
:104B8000096F200E0A6F040E0B6F880E086F040168
:104B9000280E0E6F040E0F6F400E0C6F1200D9CF4F
:104BA000E6FFE1CFD9FFE652FC0EDB50080805E234
:104BB000080EF36EFC0EF3CFDBFFDF6AFC0EDB505A
:104BC000DF5C19E2DF50E76EFD0EDBCFE9FFFE0E82
:104BD000DBCFEAFFE750E926000EEA22EF50E66E4F
:104BE000DF50EA6A280FE96E040EEA22E552E75028
:104BF000EF6EDF2AE3D7FC0EDBCF0DF4400E04018D
:104C00000C170C7D880E0C13E552E552E7CFD9FF47
:104C10001200D9CFE6FFE1CFD9FF0001F66B040106
:104C200008BF31D0FC0EDBCF02F00951D88002540E
:104C300003E2FC0E09C4DBFF0001F66BFC0EDB5047
:104C4000F65D19E2F651EA6A200FE96E040EEA22D7
:104C5000EF50E66EF651E76EFD0EDBCFE9FFFE0E7C
:104C6000DBCFEAFFE750E926000EEA22E552E750E3
:104C7000EF6EF62BE3D70401080E096F400E0817FC
:104C8000087D880E08130001F65100D0E552E7CFE9
:104C9000D9FF12006DA60CD80001ED0508E16DBA30
:104CA00006D0686A696A69806988020EED6F120031
:104CB0006D6A696A6D860001010EED6F12006D6A02
:104CC000696A0001ED6B12005FEF26F00001ED5103
:104CD00001E13AD06850040B04E06950040B01E094
:104CE0003CD86DB231D06850010B04E06950010B23
:104CF00001E054D86850100B04E06950100B01E03B
:104D000024D86850400B04E06950400B01E03BD8C8
:104D10006850200B04E06950200B01E036D8685041
:104D2000020B04E06950020B01E036D8030E0001CB
:104D3000ED5D01E209D06850080B06E06950080BF0
:104D400003E0C4EC23F068961200698468986D82D1
:104D5000A19AF290F2B005D812006D92699468940D
:104D600012000001EEA10ED0F8DF6D840001080EE4
:104D7000F76F070EF86FF707000EF85BF751F811A1
:104D8000FAE16D941200689C120070A003D02AEC26
:104D900025F07090689A1200689212006A6A686A38
:104DA0009F0E6B6E7B0E696E6E6A0F0EE66E710E55
:104DB000E66E0F0EE66E14D8E552E552E552160E79
:104DC000706E68A602D06896FCD76D982AEC25F024
:104DD0000001EE910001EF6B0001030EED6F120078
:104DE000D9CFE6FFE1CFD9FFFD0EDBCFE9FFFE0E05
:104DF000DBCFEAFFFC0EDB5004E0EE6AFC0EDB06C4
:104E0000F9D7E552E7CFD9FF1200D9CFE6FFE1CFBE
:104E1000D9FF0001040EEC6FFE0EDBA602D08D82DE
:104E200001D08D92000000000001EC078D80FE0E85
:104E3000DBCFE7FFE79EE746FE0EE7CFDBFF8D9077
:104E40000001EC51E9E1E552E7CFD9FF1200EBC0D8
:104E5000E6FFDBDFE552EAC0E6FFD7DFE552E9C057
:104E6000E6FFD3DFE552E8C0E6FFCFDFE5528D84F1
:104E70000000000000008D9412000001E86BE96B57
:104E8000EA6BEB6B27EF27F0D9CFE6FFE1CFD9FF35
:104E9000FE0EDB500F0B0001E86FFE0EDBB8D7DF14
:104EA000E552E7CFD9FF1200D9CFE6FFE1CFD9FF16
:104EB000FE0EDB500F0B0001E96FFE0EDBB8C7DF03
:104EC000E552E7CFD9FF1200D9CFE6FFE1CFD9FFF6
:104ED000FE0EDB500F0B0001EA6FFE0EDBB8B7DFF2
:104EE000E552E7CFD9FF1200D9CFE6FFE1CFD9FFD6
:104EF000FE0EDB500F0B0001EB6FFE0EDBB8A7DFE1
:104F0000E552E7CFD9FF12000001E85100D01200AE
:104F10000001E95100D012000001EA5100D0120056
:104F20000001EB5100D01200F02C52F2C8F61C5ECA
:104F30002D6D1A2A73616A293F3E3C3830202123A7
:104F4000272F475536313B4C560611150902140BD5
:104F500010041E0D1207050F161B0A08030C180E6D
:104F6000191D13682422656C17FFFFFFFFBADB7C55
:104F700092DD6DE4573E49C73EEE36D430F22BF356
:104F8000279F24CE21641F4C1D771BDA196A182134
:104F900017F915ED14FA131B134F129411E710476C
:104FA00010B20F270FA60E2D0EBC0D510DED0C8E5D
:104FB0000C350CE10B910B450BFC0AB80A770A384B
:104FC0000AFD09C4098E095A092809F808CA089E69
:104FD0000873084B082308FD07D907B60794077321
:104FE00007530734071707FA06DE06C306A9068F1C
:104FF0000676065E06470631061A060506F005DC4B
:1050000005C805B505A20590057E056D055C054B37
:10501000053B052C051C050D05FE04F004E204D437
:1050200004C704BA04AD04A004940488047C04708A
:105030000400000410801000000000082040080058
:105040000000D9CFE6FFE1CFD9FFE652C26A3C0E9D
:10505000C06EC280C282C2B2FED7C4CFF1F02D0EA4
:10506000C402F450DF6E050EDF26DFCFE6FFAAECA8
:1050700010F0E5520001F36B050EF26FCD6A9E90C1
:105080009D80D10ECF6E200ECE6ECD80E552E552C2
:10509000E7CFD9FF1200D9CFE6FFE1CFD9FFE65223
:1050A000CD909E90D10ECF6E200ECE6ECD80C2B22E
:1050B0003DD00001F151C45C04E1F36B050EF26FC9
:1050C00021D0F151C45C10E2020EF35D08E1C4503E
:1050D000F15D026E040E025C02E3F20704D0020EE0
:1050E000F36F050EF26F0ED0F30508E1F151C45CC9
:1050F000026E040E025C02E3F20704D0010EF36FAD
:10510000050EF26FF25111E12D0EC402F450DF6E64
:10511000050EDF26DFCFE6FFB6EC10F0E552C4CF78
:10512000F1F00001F36B050EF26FC28246EC15F050
:105130003EEC1FF0E552E552E7CFD9FF1200DACF7F
:10514000E4FFE2CFDAFFE9CFE4FFEACFE4FFF6CFF6
:10515000E4FFF7CFE4FFF5CFE4FFF3CFE4FFF4CFB4
:10516000E4FFFACFE4FF00EE00F0020EE80403E3F0
:10517000EECFE4FFFBD700EE02F0020EE80403E3FB
:10518000EECFE4FFFBD7E6529EA002D04BEC28F016
:10519000F050010B03E1F050020B02E019EC11F0AA
:1051A000F2A402D0D3EC12F0E55200EE03F0020EAE
:1051B000E80403E3E5CFEDFFFBD700EE01F0020EBC
:1051C000E80403E3E5CFEDFFFBD7E5CFFAFFE5CF3A
:1051D000F4FFE5CFF3FFE5CFF5FFE5CFF7FFE5CF30
:1051E000F6FFE5CFEAFFE5CFE9FFE5CFDAFF1100F3
:1051F000D8CFE4FFE0CFE4FFE46EDACFE4FFE2CF04
:10520000DAFFF3CFE4FFF4CFE4FFE652E552E5CF57
:10521000F4FFE5CFF3FFE5CFDAFFE550E5CFE0FFA0
:10522000E5CFD8FF10001201000200000008C016F0
:105230005E0601000102000109022900010100A02F
:1052400032090400000203000003092101010001EA
:105250002222000705810308000107050103080059
:1052600001040309040A034B00310058004D0012E9
:105270000353004F0032005200200042006F0078BC
:1052800000120353004F0032005200200043006F11
:10529000006E00740072006F006C006C006500729C
:1052A0000006A0FF0901A1010903150026FF0075F2
:1052B00008950281020904150026FF007508950271
:1052C0009102C038523852615265526F5281527009
:1052D0004A002A0EF66E200EF76E000EF86E0001E0
:1052E0000900F550DB6F0900F550DC6F03E1DB6767
:1052F00001D03DD00900F550D66F0900F550D76FA9
:105300000900F550D86F09000900F550E96E090051
:10531000F550EA6E090009000900F550D96F09003F
:10532000F550DA6F09000900F6CFDDF0F7CFDEF0B7
:10533000F8CFDFF0D6C0F6FFD7C0F7FFD8C0F8FF30
:105340000001D95302E1DA5307E00900F550EE6E8F
:10535000D907F8E2DA07F9D7DDC0F6FFDEC0F7FFBC
:10536000DFC0F8FF0001DB07000EDC5BBFD71200D7
:1053700007D8F28CF28E10D80FEC19F0FCD712007F
:105380000F0EC112140E6F6E0001ED6B0001EE6B7B
:105390000001EF6BF1EF18F04AEC26F06FBE02D07F
:1053A00066EC26F0120013EE00F023EE00F0F86A2F
:1053B000019C69EC29F0F6EC29F0B8EC29F0FBD758
:1053C0001200000800040002000180002000040018
:1053D000010040001000080002000002010300EE7E
:1053E00000F00F0EEE6AEA62FDD712001200000014
:1053F00000000000000000000000000000000000AD
:10540000000000000000000000000000000000009C
:10541000000000000000000000000000000000008C
:10542000FFFFFFFFFFFFFFFFFFFFFFFFFFFFFFFF8C
:0200000400F00A
:10000000012345670000008000000001FFFFFFFFA3
:10001000FFFFFFFFFFFFFFFFFFFFFFFFFFFFFFFFF0
:10002000FFFFFFFFFFFFFFFFFFFFFFFFFFFFFFFFE0
:10003000FFFFFFFFFFFFFFFFFFFFFFFFFFFFFFFFD0
:10004000FFFFFFFFFFFFFFFFFFFFFFFFFFFFFFFFC0
:10005000FFFFFFFFFFFFFFFFFFFFFFFFFFFFFFFFB0
:10006000FFFFFFFFFFFFFFFFFFFFFFFFFFFFFFFFA0
:10007000FFFFFFFFFFFFFFFFFFFFFFFFFFFFFFFF90
:10008000FFFFFFFFFFFFFFFFFFFFFFFFFFFFFFFF80
:10009000FFFFFFFFFFFFFFFFFFFFFFFFFFFFFFFF70
:1000A000FFFFFFFFFFFFFFFFFFFFFFFFFFFFFFFF60
:1000B000FFFFFFFFFFFFFFFFFFFFFFFFFFFFFFFF50
:1000C000FFFFFFFFFFFFFFFFFFFFFFFFFFFFFFFF40
:1000D000FFFFFFFFFFFFFFFFFFFFFFFFFFFFFFFF30
:1000E000FFFFFFFFFFFFFFFFFFFFFFFFFFFFFFFF20
:1000F000FFFFFFFFFFFFFFFFFFFFFFFFFFFFFF000F
:020000040020DA
:10000000FFFFFFFFFFFFFFFFFFFFFFFFFFFFFFFF00
:020000040030CA
:0E000000240E301E008181000FC00EA00F40A4
:00000001FF
